:0C2FB00033302E33202020001020304051
:082C8E00C10BC10DC10AC10F09
:102EF700758850758922758E0C758AAE758CAE757E
:062F07008BC7758DC72287
:102F0D0075A4CDE4F5F275F3F075A6E075E10675DF
:032F1D00E240226D
:102F200075BC4475E88075BA1F75D108E4F5BB43DC
:032F3000E608228E
:0C2FA40075A14075F809E4F5A2D2AE2238
:091A2400E4F5B1F5A975B28322C5
:0D2F56007592027593FE75910443E680228A
:0B2FBC0075CA8F75CBFFD2CAD2AD22C0
:1019FA00E4F5D9121A24122F0D122F20122FA41235
:081A0A002FBC122F56022EF72B
:102E4900E4FEEF30E004C2878002D287C286D286D0
:092E5900EFC313FF0EEEB402E911
:012E6200224D
:061A1B00EF04FF022E495A
:102DCD00900286E0FF121A1B900285E0FF121A1B7B
:102DDD00900284E0FF121A1B900283E0FF021A1B7F
:0228DE00A90748
:1028E000E9748729F582E43402F583E0FF7418293E
:1028F000F8E62FFBE433FAD3EB94FFEA94004004AC
:102900007A007BFF741429F8E6FD7C00AF03AE0269
:10291000121BA0AA06AB07EB7807CEC313CE13D8C1
:10292000F9FB743329F8E6FD7C00AF03121BA0AA63
:1029300006AB07EB7806CEC313CE13D8F9FBAA0675
:0F294000C2ADE925E02428F8A60208A603D2AD0F
:01294F002265
:10286A00E4FF75BB11FE75E89030EDFD742A2EF574
:10287A0082E43403F583E5BEF00E05BBEEC3940291
:10288A0040E490032AE0FED394194021A3E0FDD34B
:10289A0094194019EE94E85004C2148002D214ED3F
:1028AA00C394E85004C2138008D2138004C213C22E
:1028BA0014A214E43325E0FFA213E4334F14600B8F
:1028CA0014600B14600B24037F48227F49227F4A3D
:0428DA00227F4B22EC
:0D2F630075337F75347F75357F75367F229D
:1014BD00E4900264F01219FAE4FC12286A90030415
:1014CD00EFF00CECB40AF3900304E0FF122F7D4310
:1014DD00F601122F20122F63122E63122C65E5B028
:1014ED00541EF53730A403433701122F8A750807B0
:1014FD007509D0C20CD2AF122DCD900264E0FF6001
:10150D005330E30EE518C39403500775337FEF5442
:10151D0007F0900264E0FF30E20EE519C39403502A
:10152D000775347FEF540BF0900264E0FF30E10E4D
:10153D00E51AC39403500775357FEF540DF09002F3
:10154D0064E0FF30E00EE51BC39403500775367F52
:10155D00EF540EF0300B10900304E0FF7BFF7A2F59
:10156D0079B0122A1CC20B300D0A900304E0FF1251
:10157D002D6AC20DE524607714604724FD6019249F
:10158D00FC602224F8602B240E705E900283E00430
:10159D00F0B40302E4F08025900284E004F0B4037B
:1015AD0002E4F08018900285E004F0B40302E4F048
:1015BD00800B900286E004F0B40302E4F0122CB428
:1015CD008027300A18122F63A20CB3920C300C0630
:1015DD00C215C2A58013D2A5122F8A800CE49002E9
:1015ED0081F012300CC20FD2A5122DCDE4F52430AE
:1015FD000944C209E50945086008E50915097002A5
:10160D001508E4F508F5097D08FF1210A77D097F7F
:10161D00011210A77D0A7F021210A77D0B7F031206
:10162D0010A7E4FF1228DE7F011228DE7F021228A8
:10163D00DE7F031228DE7B017A027965122C39EFE9
:10164D007003021507900267E0121D6F16C904178B
:10165D001305168B1416781616811716901A16B2D6
:10166D001B16BD1D16C31E00001769D20CC215C274
:10167D00A5021769C20CD2A5122F8A021769D20AC8
:10168D000217697B017A027965900275EBF0A3EA86
:10169D00F0A3E9F0121B26FE900304E0FF6E600339
:1016AD000217698005900304E0FF122D8B02176964
:1016BD00122FF80217691230060217697B017A02A0
:1016CD007965900278EBF0A3EAF0A3E9F0900003BE
:1016DD00121B3FFF900304E06F6003021769300C8B
:1016ED007390027804F0A3EAF0A3E9F090000512DC
:1016FD001B3FFF900006121B3FFD900004121B3F85
:10170D00FB1226D0804E7B017A027965900278EB30
:10171D00F0A3EAF0A3E9F0900003121B3FFF900342
:10172D0004E06F7037300C2C90027804F0A3EAF0CF
:10173D00A3E9F0900005121B3FFF900006121B3F1E
:10174D00FD900004121B3FFB1224C4122C65122FB6
:10175D0097122DCD900304E0FF122E0D200C0302E5
:10176D001643900267E014603C24FA606214700323
:10177D0002182C24F97003021867240D6003021659
:10178D0043122F457B017A027965900275EBF0A328
:10179D00EAF0A3E9F0900003121B3F900281F012D2
:1017AD00300C021861122F457B017A027965900287
:1017BD0075EBF0A3EAF0A3E9F0900003121B3F9044
:1017CD000281F0122C65122F97122DCD0218611285
:1017DD002F457B017A02796590027BEBF0A3EAF04D
:1017ED00A3E9F0900003121B3FFF900004121B3F72
:1017FD00FD900005121B3FFBC00390027BE0FBA395
:10180D00E0FAA3E0F9900006121B3F900297F0D08A
:10181D000312257A122C65122F97122DCD803512B9
:10182D002F457B017A02796590027BEBF0A3EAF0FC
:10183D00A3E9F0900003121B3FFF900004121B3F21
:10184D00FD900005121B3FFB12188C122C65122FF8
:10185D0097122DCD122FDC0216437B017A0279658A
:10186D0090027EEBF0A3EAF0A3E9F0900264E0FEB3
:0F187D00C0061229B8D0E04F900264F002164363
:10240E00E5B0541EF52330A403432301E5236537BD
:10241E00600CE5236537F525753003852337E530E8
:10242E0060501530E530704AE52530E108E523208F
:10243E00E103752402E52530E208E52320E2037569
:10244E002404E52530E308E52320E303752408E59D
:10245E002530E408E52320E403752410E52530E05B
:10246E0011E52320E00C900302740FF0A374A0F08A
:10247E00D20E300E29900303E024FFF0900302E009
:10248E0034FFF0E5A030E405752401C20E9003027E
:10249E00E07002A3E07007C20E300A02D20BE51301
:1024AE0045126011E51315137002151214451270C2
:0624BE0004C2A6C2A72221
:03301E00D2FA22C1
:102F33008532A39002FF74FFF0A37430F0A3741ED4
:022F4300F0227A
:102EC900C2FAE5314527F5A39002FF74FFF0A37418
:072ED9002FF0A37433F02277
:031A1500022AC8DA
:102AC800C0E0C0F0C083C082C0D075D000C000C0D4
:102AD80001C002C003C004C005C006C007C2FF9001
:102AE80002FFA3E0FAA3E0F9121D95D007D006D0A3
:102AF80005D004D003D002D001D000D0D0D082D0ED
:062B080083D0F0D0E032A2
:031A120002295056
:10295000C0E0C083C082C0D075D000C000C006C037
:1029600007C2CFE52625E02428F8E6FE08E625E0A4
:10297000FFEE33FE74A72FF58274083EF583E493CF
:10298000F531740193F532E526902FB893F52705BC
:1029900026E526B404037526009002FF74FFF0A319
:1029A000742EF0A374C9F0D2FFD007D006D000D0A7
:0829B000D0D082D083D0E032C8
:031A2D00022E2C5A
:102E2C00C0E0C083C082C0D053917F12240E75E8DD
:0D2E3C009075BB01D0D0D082D083D0E032A1
:031A2100022B99FC
:102B9900C0E0C0D075D000C000C007C2EDE5BB6081
:102BA90019AFBB74132FF8A6BE75E890E5BBB40B3B
:102BB9000575BB00800905BB800585BE1FD209D0FC
:082BC90007D000D0D0D0E032AB
:082C9600410282044102930097
:06300600E4900293F022A9
:072FF8009002937401F02226
:10262C009003207404F0E4A3F0FFA3F0A37408F06B
:10263C00E4A3F0122FF07E3A7F007B017A0379201D
:10264C00900312E4F0A304F0122B0E122CDAE4FF28
:10265C0074872FF582E43402F583E4F00FEFB404B1
:10266C00EFE4900283F0A3F0A3F0A3F0900321F029
:10267C00900321E0FFC3941E502FEF75F008A424A3
:10268C0001F582E4343AAF82FE7B017A02798390C1
:10269C000322E0FDA3E0900312CDF0A3EDF0122B8A
:1026AC000E900321E004F080C7122CDA7E3A7FF101
:1026BC007B017A037924900312E4F0A304F0122B2B
:0426CC000E022CDAF4
:102CB400900282E0600414F0800B200A08200F05C3
:102CC400D20F53A0DF20150D300C0A900293E07050
:062CD40002D20DD2152210
:102E6300903AF1E493F46009903A00E493640460C7
:0A2E73000312262CE4900281F022E5
:102C6500900281E0FFC3941E501EEF75F008A42466
:102C750001F9743A35F0FA7BFF78837C027D017E99
:092C8500007F08121B00C2152299
:102BD100900281E0C3941E502A122FF0900281E0EE
:102BE10075F008A42401F582E4343AAF82FE7B013A
:102BF1007A027983900312E4F0A37408F0122B0E89
:042C0100122CDA2295
:06300C00122BD1C21522B7
:05257A00900295EDF058
:10257F00900297E004F090029AEFF0A3EBF0900234
:10258F0095E0FF90029AE0FED39F400302262BEEC8
:10259F0075F008A42401F582E4343AAF8290029CCE
:1025AF00F0A3EFF090029BE075F008A42401F582F0
:1025BF00E4343AAF8290029EF0A3EFF0E4900298D9
:1025CF00F0A3F090029EE475F001121BC8AFF0FE6D
:1025DF0090029CE0FCA3E0F5828C83E493FD12272C
:1025EF006590029DE004F0700690029CE004F0906C
:1025FF000299E004F07006900298E004F0C3900294
:10260F0099E09408900298E0940040B7122CDA9069
:0C261F00029AE004F0A3E004F002258D14
:01262B00228C
:05188C009002D4EDF014
:101891009002D9EFF0A3EBF09002D4E0FF9002D9CF
:1018A100E0D39F40030219F9A3E075F008A42401D5
:1018B100F582E4343AAF829002D5F0A3EFF0E490E0
:1018C10002DBF0A3F09002DBE0FEA3E0FFC394088B
:1018D100EE940050389002D5E0FCA3E0F5828C83B1
:1018E100E493FD748B2FF582E43402F583EDF090DF
:1018F10002D6E004F070069002D5E004F09002DC1C
:10190100E004F070C09002DBE004F080B89002D9EE
:10191100E075F008A42401F582E4343AAF82900224
:10192100D7F0A3EFF09002DAE075F008A42401F5F6
:1019310082E4343AAF829002D5F0A3EFF0E4900252
:10194100DBF0A3F09002D5E475F001121BC8AFF0F3
:10195100FE9002D7E0FCA3E0F5828C83E493FD12B4
:1019610027659002D8E004F070069002D7E004F0F9
:101971009002DCE004F070069002DBE004F0C3901A
:1019810002DCE094089002DBE0940040B79002D9B9
:10199100E075F008A42401F582E4343AAF829002A4
:1019A100D7F0A3EFF0E49002DBF0A3F09002DBE0CC
:1019B100FCA3E0FDC39408EC9400502C9002D7E402
:1019C10075F001121BC8AFF0FE748B2DF582E43463
:1019D10002F583E0FD1227659002DCE004F070CC93
:1019E1009002DBE004F080C4122CDA9002D9E0040A
:0819F100F0A3E004F0021899D4
:0119F90022CB
:0B24C4009002B6EFF0A3EDF0A3EBF0E8
:1024CF00A2AFE433A3F0C2AF122FFF9002B7E0FE2A
:1024DF009002B6E0FDEDFF9002BEEEF0A3EFF0E448
:1024EF009002BAF09002B8E0FF9002BEE0FCA3E0C9
:1024FF00FD7B017A02798B9002F5E4F0A37408F06A
:10250F00122D489002BFE02408F09002BEE0340084
:10251F00F09002BAE075F008A42401F9743A35F08E
:10252F00FAA374FFF0A3EAF0A3E9F0122FF09002E0
:10253F00BBA3E0FAA3E0AE02FF7B017A02798B9096
:10254F000312E4F0A37408F0122B0E122CDA90028F
:10255F00BAE004F0E0C3941E408A900304E0FF1237
:0A256F002F7D9002B9E024FF92AF27
:01257900223F
:0B26D0009002DDEFF0A3EDF0A3EBF0B3
:1026DB00A2AFE433A3F0C2AF122FFF9002DEE0FEF5
:1026EB009002DDE0FDEDFF9002E2EEF0A3EFF0E4EF
:1026FB009002E1F09002E1E0FFC3941E504BEF75A6
:10270B00F008A42401F582E4343AAF82FE9002E48F
:10271B00F0FAA3EFF0FB9002DFE0FF9002E2E0FCA7
:10272B00A3E0FDA9037BFF9002FDE4F0A37408F086
:10273B00122E979002E3E02408F09002E2E03400BE
:10274B00F09002E1E004F080AB900304E0FF122F65
:09275B007D9002E0E024FF92AF42
:012764002252
:0E2B5400900314EBF0A3EAF0A3E9F0A3EDF078
:102B6200E4900319F0900314E0FBA3E0FAA3E0F968
:102B7200A3E090030AF0900318E090030BF0E4FF47
:102B82001227F1EFB4FF0D900319E0FE04F0EEC33B
:062B9200940340D17E0017
:012B9800221A
:0B2C3900900342EBF0A3EAF0A3E9F0E7
:102C44007E007F007D10121D9B900342E0FBA3E0F9
:102C5400FAA3E0F97D101221FCEF7002FF227F013C
:012C6400224D
:102A1C009002C07422F0A3EFF0A37413F0121B26E3
:102A2C009002C3F0900001121B3F9002C4F0900082
:102A3C0002121B3F9002C5F0900003121B3F900244
:102A4C00C6F0900004121B3F9002C7F090000512D4
:102A5C001B3F9002C8F0900006121B3F9002C9F079
:102A6C007B017A0279C0E4900318F07D0A022B54A2
:102D6A0090032E7422F0A3EFF0A37403F0A374FF70
:102D7A00F07B017A03792EE4900318F07D04022B8C
:012D8A0054F4
:102D8B009003327422F0A3EFF0A3741CF0A374FF32
:102D9B00F07B017A037932E4900318F07D04022B67
:012DAB0054D3
:102E0D00E4900336F0A3EFF0A3740AF0A3EFF07B88
:0F2E1D00017A037936E4900318F07D04022B54F8
:102C9E00420262000042020D00004202080000C122
:052CAE0012C111C1106C
:0A2FD200C211C212E490020CF022BA
:102D2500E4900262F0A3F090020DF0A3F0A3F090FE
:102D35000208F0A3F0900203F0A37440F0E49002BF
:032D45000BF0226E
:06301200122FD2022D2551
:0D2F700075C19043E60190020A7401F02241
:102F450043C140E5C120E5FB123012E490020AF0CE
:012F55002259
:0A2FDC0053C1BF90020A7401F022F5
:0D2F7D00AE07122F70900207EEF002301226
:102D0000E4900345F0A3F0301102FF222012FDD21F
:102D100011900205E4F0A37410F0900250EFF0E47B
:042D2000A3F07F019C
:012D2400228C
:102C050030110A900205E07002A3E070037F0022F4
:102C1500900206E024FFF0900205E034FFF09002F8
:102C250051E0FE04F074522EF582E43402F583EF90
:042C3500F07F012209
:0B2FC700301107C211D212122FE622B7
:0A2FE600E5C120E5FBC2C4D2C522FC
:1027F100900307EBF0A3EAF0A3E9F090020AE0707E
:1028010002FF2290030AE0FE6005D3941040037F8B
:082811000022122D00EF604EC1
:10281900E490030CF090030AE0FF90030CE0FEC380
:102829009F5024900307E0FBA3E0FAA3E0F98E820E
:10283900758300121B3FFF122C05EF7002FF2290D7
:10284900030CE004F080CEE490020CF0122FC79044
:0E285900030BE070032012FD90020CE0FF2242
:032867007FFF22CE
:0E21FC0090033AEBF0A3EAF0A3E9F0A3EDF0B4
:10220A00E4FFD3900263E09400900262E064809459
:10221A008050012253E6FE900208E0FEA3E0240F5C
:10222A00F58274023EF583E0FF900208E475F0013E
:10223A00121BB2FCE5F064404C7006900208F0A351
:10224A00F0900204E004F07006900203E004F0E467
:10225A00FE90033DE0FDEEC39D5054EEC39F504FE8
:10226A00900208E0FCA3E0240FF58274023CF58397
:10227A00E0FD90033AE0FBA3E0FAA3E0F98E827551
:10228A008300ED121B7E900208E475F001121BB266
:10229A00FCE5F064404C7006900208F0A3F090024E
:1022AA0004E004F07006900203E004F00E80A2EE4F
:1022BA00C39F5029900208E475F001121BB2FCE595
:1022CA00F064404C7006900208F0A3F0900204E01B
:1022DA0004F07006900203E004F00E80D2900263CC
:1022EA00E024FFF0900262E034FFF043E60190033D
:0C22FA003DE0FEEFC39E50028002AF06E4
:0123060022B4
:102EB100D3900263E09400900262E06480948040C9
:082EC100047F0180027F002262
:031A1800021DC7E5
:101DC700C0E0C0F0C083C082C0D075D000C000C0E2
:031DD70006C0073C
:101DDA00C217E5C054FE121D6F1EB6081EB60A1EB3
:101DEA007D0C1E7D0E1F2F101F2F121E83221E8E8A
:101DFA00281E8E2A1E832C1E832E1E70C01E29C2E8
:101E0A001E14E01E14E200001F3AC210900250E0B5
:101E1A00F5C2C2C5C2C490024F74FFF0021F3C90C3
:101E2A00024FE0FFB4FF12900251E0F5C2C2C5C2F0
:101E3A00C490024FE4F0021F3C900251E0FEEFC34F
:101E4A009E501790024FE0FF04F074522FF582E47F
:101E5A003402F583E0F5C2021F3CD2C490020CE4BE
:101E6A00F0C212021F3C90020C74FDF0D2C5C2C42B
:101E7A00021F3C90024F74FFF0D210C2C4C2C1D2FA
:101E8A00C5021F3CE5C26007900207E0B5C20E908A
:101E9A000202E4F0C2C5C2C4D2C1021F3CC2C4C21B
:101EAA00C1301003021F34C2C5021F3C900202E077
:101EBA007020E5C2F0E0FFC3900204E09F7480F84E
:101ECA00900203E06480985003122D25900202E0EC
:101EDA0004F0900204E024FFF0900203E034FFF0E3
:101EEA0090020DE0FEA3E0240FF58274023EF58312
:101EFA00E5C2F090020DE475F001121BB2FEE5F0A6
:101F0A0064404E700690020DF0A3F0900202E014B5
:101F1A00F0700E900263E004F07006900262E00432
:101F2A00F0D2C1800DC2C4301008C210D2C58002DE
:101F3A00D21730171053C17F43C180C2C5C2C4C271
:071F4A00C1C217C212C2C0A0
:101F5100D007D006D000D0D0D082D083D0F0D0E04E
:011F6100324D
:05301800E5C15420FF9A
:01301D002290
:072FFF0043C14053E6FE222E
:101F62009002E6E0FFA3E0FCA3E0FDA3E0FBA3E018
:101F7200FAA3E0F99002A6E538F0E539A3F0900261
:061F8200EEE09002A8F061
:101F88009002A0EFF0A3ECF0A3EDF0A3EBF0A3EA2E
:041F9800F0A3E9F0D9
:101F9C009002A97403F0A374E8F0E5C120E5FBD22C
:101FAC00C1C2C4D2C5E4FF900348F030C0FDE5C007
:101FBC0054FE2440700302205F24FE602424E2605F
:101FCC000924FE600524E2022067C2C5EF6003020B
:101FDC00206D9002A0E025E044A0F5C27F03022012
:101FEC006DEFB4030A9002A1E0F5C27F058072EF99
:101FFC00B4050B9002A1A3E0F5C27F068063EF64E9
:10200C0006703E9002A8E09002A3700FE0FBA3E4E0
:10201C0075F001121BC8A9F0FA8008E0FBA3E0FAE6
:10202C00A3E0F9121B26F5C29002A7E024FFF09062
:10203C0002A6E034FFF0E07002A3E070247F07807A
:10204C0020EFB40706D2C47F0980169003487405AC
:10205C00F0800E9003487402F080069003487401DF
:10206C00F0EFB40904C2C08036900348E0FE640669
:10207C006012EEB402169002A974FFF5F0121BB2B6
:10208C0045F06008D2C5E4900348F0FF900348E0A7
:10209C006008C2C5D2C4C2C08005C2C0021FB7E569
:0420AC00C120E5FB6F
:0120B000220D
:1020B1009002CAEFF0A3ECF0A3EDF0A3EBF0A3EADA
:0420C100F0A3E9F0AF
:1020C5009002D27403F0A374E8F0E5C120E5FBD2D9
:1020D500C1C2C4D2C5E4FF900348F030C0FDE5C0DD
:1020E50054FE24C870030221A224AE607A24CA706B
:1020F500030221AA24FE603824E2600924FE60055B
:1021050024E20221B2C2C5EF700F9002CAE025E0B9
:1021150044A0F5C27F030221B8EF640160030221E8
:10212500B89002CAE025E044A1F5C27F040221B8B7
:10213500EFB4030A9002CBE0F5C27F058075EFB4DA
:10214500050B9002CBA3E0F5C27F068066EFB406CF
:1021550006D2C57F01805CEFB404047F02805490F1
:1021650003487405F0804C9002CDE0FBA3E475F0C4
:1021750001121BC8A9F0FAE5C2121B6C9002D1E04E
:1021850024FFF09002D0E034FFF0E07002A3E0708D
:10219500087F09C2C1D2C4801A7F02801690034805
:1021A5007406F0800E9003487402F0800690034890
:1021B5007401F0EFB40904C2C08036900348E0FE14
:1021C50064066012EEB402169002D274FFF5F012A6
:1021D5001BB245F06008D2C5E4900348F0FF9003B8
:1021E50048E06008C2C5D2C4C2C08005C2C0022092
:0621F500E0E5C120E5FB5E
:0121FB0022C1
:102307009002E6EFF09002E9EBF0A3EAF0A3E9F020
:082317009002E7ECF0A3EDF0E9
:10231F00753A00543FF53B543F605CC37440953BA6
:10232F00FFE4953AFE9002ECE0FCA3E0FDC39FECC6
:10233F009E50068C388D3980048E388F39121F626B
:10234F00900348E060037F02229002E8E02539F015
:10235F009002E7E03538F09002EEE0700B9002EA61
:10236F00E5388539F0121BB2C39002EDE09539F0D4
:10237F009002ECE09538F09002ECE0F538A3E0F530
:10238F0039D3E5399400E53894004070E53994402D
:10239F00E53894005013121F62900348E060037FEA
:1023AF000222E4F538F53980D89002E6E0FFA3E089
:1023BF00FCA3E0FDA3E0FBA3E0FAA3E0F99002A6E3
:1023CF00E4F07440121F7E900348E060037F022206
:1023DF0074C02539F53974FF3538F5389002E8E0C7
:1023EF002440F09002E7E03400F09002EEE07091AC
:0E23FF009002EA75F040121BB20223907F009C
:01240D0022AC
:102EE0009002D0E4F0A304F01220B1900348E06017
:072EF000037F01227F002295
:102E7D00900347EBF07B017A0379479002ECE4F085
:0A2E8D00A304F0E4A3F012230722CF
:102D4800C0079002F5E0FFA3E09002D0CFF0A3EF18
:102D5800F0D0071220B1900348E060037F01227F82
:022D6800002247
:102E9700C0079002FDE0FFA3E09002ECCFF0A3EFA4
:0A2EA700F0E4A3F0D0071223072285
:102DAC00A2AFE433FCC2AF758F0175B7A575B7F14F
:102DBC008F828E83EDF0E4F58FAF04EF24FF92AF9A
:012DCC0022E4
:102DED00A2AFE433FDC2AF758F0375B7A575B7F10B
:0F2DFD008F828E83E4F0F58FAF05EF24FF92AF46
:012E0C0022A3
:102A7C0090033EEEF0A3EFF0A3ECF0A3EDF0EB4AE5
:102A8C00603990033EE0FEA3E0FFA3E0FCA3E0F579
:102A9C00828C83E0FD122DACEB1B70011A9003416C
:102AAC00E004F07006900340E004F090033FE00473
:0C2ABC00F070CB90033EE004F080C322D9
:082FF000E4900000F0A3F022C0
:102CDA00900000E0FEA3E0FF122DED900000E0FE60
:102CEA00A3E0FF7C007D027B007A02122A7CE4903A
:062CFA000000F0A3F0222F
:0A276500A90590031AEEF0A3EFF0AF
:10276F00EE54FEFE900000E0FCA3E0FD7002EE6C64
:10277F006057ED4C6003122CDA90031AE0FEEE5412
:10278F00FEFE7F00900000F0A3EFF090031CEEF030
:10279F00A3EFF0A37400F0A37402F07E0290031C69
:1027AF00E475F001121BC885F082F583E493FD9068
:1027BF00031EE475F001121BC885F082F583EDF05E
:1027CF00EF1F70011EEF4E70D490031AE0FCA3E0D0
:1027DF00FDEC5401FC74022DF58274003CF583E985
:0127EF00F0F9
:0127F00022C6
:102B0E0090030DEEF0A3EFF0A3EBF0A3EAF0A3E930
:102B1E00F090031274FFF5F0121BC845F06026907A
:102B2E00030DE475F001121BC8AFF0FE90030FE029
:102B3E00FBA3E475F001121BC8A9F0FA121B26FDC7
:062B4E0012276580CC2275
:1008A7000000000000000000000000040004000435
:1008B700000400040004000400040004000400080D
:1008C70000080008000800080008000800080008E1
:1008D7000008000C000C000C000C000C000C000CB5
:1008E700000C000C000C001000100010001000108D
:1008F7000010001000100010001000140014001465
:10090700001400140014001400140014001400183C
:100917000018001800180018001800180018001810
:100927000018001C001C001C001C001C001C001CE4
:10093700001C001C001C00200020002000200020BC
:100947000020002000200020002000240024002494
:10095700002400240024002400240024002400286C
:100967000028002800280028002800280028002840
:100977000028002C002C002C002C002C002C002C14
:10098700002C002C002C00300030003000300030EC
:1009970000300030003000300030003400340034C4
:1009A700003400340034003400340034003400389C
:1009B7000038003800380038003800380038003870
:1009C7000038003C003C003C003C003C003C003C44
:1009D700003C003C003C004000400040004000401C
:1009E70000400040004000400040004400440044F4
:1009F70000440044004400440044004400440048CC
:100A0700004800480048004800480048004800489F
:100A17000048004C004C004C004C004C004C004C73
:100A2700004C004C004C005000500050005000504B
:100A37000050005000500050005000540054005423
:100A470000540054005400540054005400540058FB
:100A570000580058005800580058005800580058CF
:100A67000058005C005C005C005C005C005C005CA3
:100A7700005C005C005C006000600060006000607B
:100A87000060006000600060006000640064006453
:100A9700006400640064006400640064006400682B
:100AA70000680068006800680068006800680068FF
:100AB7000068006C006C006C006C006C006C006CD3
:100AC700006C006C006C00700070007000700070AB
:100AD7000070007000700070007000740074007483
:100AE700007400740074007400740074007400785B
:100AF700007800780078007800780078007800782F
:100B07000078007C007C007C007C007C007C007C02
:100B1700007C007C007C00800080008000800080DA
:100B270000800080008000800084008400840084AE
:100B37000084008400840084008400840088008886
:100B4700008800880088008800880088008800885E
:100B5700008C008C008C008C008C008C008C008C2E
:100B6700008C009000900090009000900090009002
:100B770000900090009000940094009400940094DA
:100B870000940094009400940098009800980098AE
:100B9700009800980098009800980098009C009C86
:100BA700009C009C009C009C009C009C009C00A05A
:100BB70000A000A000A000A000A000A000A000A02E
:100BC70000A400A400A400A400A400A400A400A4FE
:100BD70000A400A800A800A800A800A800A800A8D2
:100BE70000A800A800AC00AC00AC00AC00AC00ACA6
:100BF70000AC00AC00B000B000B000B000B000B076
:100C070000B000B000B000B400B400B400B400B449
:100C170000B400B400B400B800B800B800B800B819
:100C270000B800B800B800BC00BC00BC00BC00BCE9
:100C370000BC00BC00BC00C000C000C000C000C0B9
:100C470000C000C000C000C400C400C400C400C489
:100C570000C400C400C800C800C800C800C800C855
:100C670000C800CC00CC00CC00CC00CC00CC00CC21
:100C770000D000D000D000D000D000D000D000D4E9
:100C870000D400D400D400D400D400D400D800D8B5
:100C970000D800D800D800D800DC00DC00DC00DC7D
:100CA70000DC00DC00E000E000E000E000E000E045
:100CB70000E400E400E400E400E400E400E800E805
:100CC70000E800E800E800E800EC00EC00EC00ECCD
:100CD70000EC00F000F000F000F000F000F400F489
:100CE70000F400F400F400F400F800F800F800F84D
:100CF70000FC00FC00FC00FC00FC010001000100FE
:100D070001000100010401040104010401080108B4
:100D1700010801080108010C010C010C010C01106C
:100D2700011001100110011401140114011401181C
:100D3700011801180118011C011C011C011C0120CC
:100D47000120012001240124012401240128012874
:100D57000128012C012C012C012C0130013001301C
:100D6700013401340134013801380138013C013CB8
:100D7700013C013C0140014001400144014401485C
:100D870001480148014C014C014C015001500150F0
:100D970001540154015801580158015C015C015C80
:100DA7000160016001640164016401680168016C0C
:100DB700016C017001700170017401740178017890
:100DC700017C017C0180018001800184018401880C
:100DD7000188018C018C0190019001940194019884
:100DE7000198019C019C01A001A401A401A801A8EC
:100DF70001AC01AC01B001B001B401B801B801BC4C
:100E070001BC01C001C401C401C801C801CC01D0A3
:100E170001D001D401D801D801DC01DC01E001E4F3
:100E270001E801E801EC01F001F001F401F801F833
:100E370001FC0200020402040208020C0210021064
:100E470002140218021C0220022002240228022C8B
:100E57000230023002340238023C024002440248A7
:100E6700024C024C025002540258025C02600264B7
:100E77000268026C027002740278027C02800284AB
:100E87000288028C029002940298029C02A002A49B
:100E970002A802AC02B002B802BC02C002C402C877
:100EA70002CC02D002D802DC02E002E402EC02F03B
:100EB70002F402F802FC03040308030C03140318EA
:100EC700031C03240328032C03340338034003447F
:100ED700034803500354035C03600368036C037403
:100EE700037803800384038C03900398039C03A473
:100EF70003AC03B003B803C003C403CC03D403D8C3
:100F070003E003E803F003F403FC0404040C0414F3
:100F1700041804200428043004380440044804500A
:100F270004580460046804700478048004880490FA
:100F3700049804A004A804B004B804C404CC04D4DE
:100F470004DC04E804F004F80500050C0514051C8E
:100F570005280530053C0544054C05580560056C1A
:100F670005740580058C059405A005A805B405C082
:100F770005C805D405E005EC05F40600060C0618BF
:100F870006240630063806440650065C06680674D2
:100F97000680068C069806A806B406C006CC06D8B6
:100FA70006E406F40700070C071C07280734074464
:100FB70007500760076C077C0788079807A407B4E2
:100FC70007C407D007E007F007FC080C081C082C2B
:100FD700083C084C085C086808780888089C08AC36
:100FE70008BC08CC08DC08EC08FC0910092009300B
:100FF70009440954096409780988099C09AC09C09E
:1010070009D409E409F80A0C0A1C0A300A440A58E8
:101017000A6C0A800A940AA80ABC0AD00AE40AF8E9
:101027000B0C0B200B340B4C0B600B740B8C0BA0B5
:101037000BB80BCC0BE40BF80C100C280C3C0C5425
:101047000C6C0C840C9C0CB40CCC0CE40CFC0D1438
:101057000D2C0D440D5C0D780D900DA80DC40DDC05
:101067000DF80E100E2C0E440E600E7C0E940EB072
:101077000ECC0EE80F040F200F3C0F580F740F9083
:101087000FB00FCC0FE80FFC0FFC0FFC0FFC0FFC91
:101097000FFC0FFC0FFC0FFC0FFC0FFC0FFC0FFCF1
:0D2F8A00D204D203D202D201C2A6C2A722F5
:0D2F9700C204C203C202C201C2A6C2A72228
:0710A7009002ABEFF0AB0576
:1010AE00C2AFC200E0FF240AF8E6900329F0FD74F7
:1010BE00142BF8E6F9C39DFCE494009002ACF0A367
:1010CE00CCF030054D9002ACE0FCA3E0FDC3EC6427
:1010DE00809480502E740E2FF8E6700276039002E4
:1010EE00ABE0FF240EF816E66003021183740E2F98
:1010FE00F8760174142BF8E6FE740A2FF8A606D2C1
:10110E00008072D3ED9404EC64809480405EC2053E
:10111E00804D9002ACE0FEA3E0FFD39400EE64801D
:10112E009480402E9002ABE0240EF8E67002760317
:10113E009002ABE0FD240EF816E67039740E2DF811
:10114E00760174142BF8E6FC740A2DF8A604D2006E
:10115E008023C3EF94FCEE6480947F500FD20590F1
:10116E0002ABE0240AF8A601D20080099002ABE09F
:10117E00240EF8E4F6E509450860030214BA2000CF
:10118E00030214BA9002ABE0FD2487F582E4340228
:10119E00F583E0FE74252DF582E43403F583E0FD3E
:1011AE00EDFFE4FCFD9002AE121D329002ACE0FEAB
:1011BE00A3E0FFD39400EE6480948050030212DD0E
:1011CE00EE3395E0FDFC7810121D1F9002B2121D39
:1011DE00329002B2E0FCA3E0FDA3E0FEA3E0FFC06C
:1011EE0006C007900329E0FFC374FF9FFFE494003D
:1011FE00AB07FAE4F9F8D007D006121C699002B2D8
:10120E00121D329002B2E0F8A3E0F9A3E0FAA3E0D7
:10121E00FB9002ABE02487F582E43402F583E0FF15
:10122E00C374FF9FFFE49400FEE4FCFD121BDE90EE
:10123E0002B2121D329002ABE02487F582E4340232
:10124E00F583E0FF900329E0D39F9002B2E0FCA368
:10125E00E0FDA3E0FEA3E0FFE440067B407A0180C0
:10126E00037BC0FAF9F8121BDE9002B2121D329007
:10127E0002AEE0F8A3E0F9A3E0FAA3E0FBC000A3FE
:10128E00E0FCA3E0FDA3E0FEA3E0FF7810121D0C2E
:10129E00D000EB2FFFEA3EFEE93DFDE83CFC90025C
:1012AE00AE121D32E47FFF7EFFFDFC9002AEE0F831
:1012BE00A3E0F9A3E0FAA3E0FBD3121CFB50030258
:1012CE0013F39002AE121D3E0000FFFF0213F390C7
:1012DE0002ACE0FEA3E0FFC3E49FFFE49EFE339565
:1012EE00E0FDFC7810121D1F9002B2121D3290020A
:1012FE00B2E0FCA3E0FDA3E0FEA3E0FFC007900375
:10130E0029E0FBE4FAF9F8D007121C699002B21238
:10131E001D329002B2E0F8A3E0F9A3E0FAA3E0FBDD
:10132E009002ABE02487F582E43402F583E0FFE41B
:10133E00FCFDFE121BDE9002B2121D329002ABE0DB
:10134E002487F582E43402F583E0FF900329E0C39D
:10135E009F9002B2E0FCA3E0FDA3E0FEA3E0FFE459
:10136E0050067B407A0180037BC0FAF9F8121BDE2F
:10137E009002B2121D329002AEE0FCA3E0FDA3E09B
:10138E00FEA3E0FFC004C005C006C007A3E0FCA397
:10139E00E0FDA3E0FEA3E0FF7810121D0CA804A947
:1013AE0005AA06AB07D007D006D005D004C3EF9B25
:1013BE00FFEE9AFEED99FDEC98FC9002AE121D32F6
:1013CE00E47FFF7EFFFDFC9002AEE0F8A3E0F9A300
:1013DE00E0FAA3E0FBD3121CFB400A9002AE121DF2
:1013EE003E000000009002AEA3A3A3E0FF9002AB6C
:1013FE00E0FB2425F582E43403F583EFF09002AE92
:10140E00E0FCA3E0FDA3E0FEA3E0FF7808121D0CB4
:10141E009002AE121D3274872BF582E43402F583EE
:10142E00E0FFE4FCFDFE9002AEE0F8A3E0F9A3E0DD
:10143E00FAA3E0FBC3121CFB601A9002AEA3A3A397
:10144E00E0FF9002ABE02487F582E43402F583EFEF
:10145E00F0122CB430052E9002ABE0FF240AF8E611
:10146E00FE2404FDE433FC74872FF582E43402F588
:10147E0083E0FFD39DEC6480F8748098502EEFC308
:10148E009E402980239002ABE0FF240AF8E6FE740A
:10149E00872FF582E43402F583E0FFD39E500DEEE4
:0E14AE0024FCFEEFC39E4004C2A6C2A7D2AF2C
:0114BC00220D
:1029B800900003121B3FFF540FFEE4FDEF54F06438
:0329C80090703CD0
:1029CB00900006121B3F900349F0900304E064480B
:1029DB00703CEE30E306900349E0F533EE30E2064F
:1029EB00900349E0F534EE30E106900349E0F5350C
:0A29FB00EE30E01A900349E0F536D3
:102A05008012EF54F0FFBF800B900304E0B448043C
:062A1500AF06AD07AF059E
:012A1B002298
:03000000020800F3
:03000300021A03DB
:03000B00021A06D0
:03001300021A09C5
:03001B00021A0CBA
:03002300021A0FAF
:03002B00021A12A4
:03003300021A1599
:03003B00021A188E
:03004300021A1B83
:03004B00021A1E78
:03005300021A216D
:03005B00021A2462
:03006300021A2757
:03006B00021A2A4C
:03007300021A2D41
:10080000E4F5D9E5EF7480F5FF7402F5EF787FE445
:10081000F6D8FD9000007F007E04E4F0A3DFFCDE4C
:07082000FA75813B0208623A
:100827000214BDE493A3F8E493A34003F68001F216
:1008370008DFF48029E493A3F85407240CC8C333D2
:10084700C4540F4420C8834004F456800146F6DFA1
:10085700E4800B0102040810204080902C8EE47E77
:10086700019360BCA3FF543F30E509541FFEE49396
:10087700A360010ECF54C025E060A840B8E493A35D
:10088700FAE493A3F8E493A3C8C582C8CAC583CA88
:10089700F0A3C8C582C8CAC583CADFE9DEE780BE40
:012CB3000020
:101A3000E709F608DFFA8046E709F208DFFA803E98
:101A400088828C83E709F0A3DFFA8032E309F60885
:101A5000DFFA8078E309F208DFFA807088828C83ED
:101A6000E309F0A3DFFA806489828A83E0A3F608A1
:101A7000DFFA805889828A83E0A3F208DFFA804C7B
:101A800080D280FA80C680D4806980F28033801052
:101A900080A680EA809A80A880DA80E280CA8033BB
:101AA00089828A83ECFAE493A3C8C582C8CCC58333
:101AB000CCF0A3C8C582C8CCC583CCDFE9DEE78003
:101AC0000D89828A83E493A3F608DFF9ECFAA9F082
:101AD000EDFB2289828A83ECFAE0A3C8C582C8CCD8
:101AE000C583CCF0A3C8C582C8CCC583CCDFEADEF1
:101AF000E880DB89828A83E493A3F208DFF980CC53
:101B000088F0EF60010E4E60C388F0ED2402B4044B
:101B10000050B9F582EB2402B4040050AF232345F2
:061B20008223901A80737D
:101B2600BB010689828A83E0225002E722BBFE02BD
:091B3600E32289828A83E49322F0
:101B3F00BB010CE58229F582E5833AF583E022505B
:101B4F0006E92582F8E622BBFE06E92582F8E222A5
:0D1B5F00E58229F582E5833AF583E49322BF
:101B6C00BB010689828A83F0225002F722BBFE0158
:021B7C00F32252
:101B7E00F8BB010DE58229F582E5833AF583E8F09D
:101B8E00225006E92582C8F622BBFE05E92582C849
:021B9E00F22231
:101BA000EF8DF0A4A8F0CF8CF0A428CE8DF0A42E59
:021BB000FE2213
:101BB200C5F0F8A3E028F0C5F0F8E58215827002BE
:061BC2001583E038F0225B
:101BC800A3F8E0C5F025F0F0E582158270021583D0
:061BD800E0C838F0E8222D
:101BDE00E88FF0A4CC8BF0A42CFCE98EF0A42CFCA6
:101BEE008AF0EDA42CFCEA8EF0A4CDA8F08BF0A424
:101BFE002DCC3825F0FDE98FF0A42CCD35F0FCEB83
:101C0E008EF0A4FEA9F0EB8FF0A4CFC5F02ECD3947
:0F1C1E00FEE43CFCEAA42DCE35F0FDE43CFC22B4
:101C2D0075F008758200EF2FFFEE33FECD33CDCC6E
:101C3D0033CCC58233C5829BED9AEC99E5829840F1
:101C4D000CF582EE9BFEED9AFDEC99FC0FD5F0D6CE
:101C5D00E4CEFBE4CDFAE4CCF9A88222B800C1B9F8
:101C6D000059BA002DEC8BF084CFCECDFCE5F0CB36
:101C7D00F97818EF2FFFEE33FEED33FDEC33FCEB6F
:101C8D0033FB10D703994004EB99FB0FD8E5E4F92A
:101C9D00FA227818EF2FFFEE33FEED33FDEC33FC17
:101CAD00C933C910D7059BE99A4007EC9BFCE99A0B
:101CBD00F90FD8E0E4C9FAE4CCFB2275F010EF2F50
:101CCD00FFEE33FEED33FDCC33CCC833C810D70750
:101CDD009BEC9AE899400AED9BFDEC9AFCE899F88B
:0E1CED000FD5F0DAE4CDFBE4CCFAE4C8F9221E
:101CFB00EB9FF5F0EA9E42F0E99D42F0E89C45F03F
:011D0B0022B5
:101D0C00E8600FECC313FCED13FDEE13FEEF13FFB5
:031D1C00D8F122D9
:101D1F00E8600FEFC333FFEE33FEED33FDEC33FC22
:031D2F00D8F122C6
:0C1D3200ECF0A3EDF0A3EEF0A3EFF02224
:101D3E00A8828583F0D083D082121D55121D5512B4
:101D4E001D55121D55E473E493A3C583C5F0C583D9
:101D5E00C8C582C8F0A3C583C5F0C583C8C582C8EF
:011D6E002252
:101D6F00D083D082F8E4937012740193700DA3A303
:101D7F0093F8740193F5828883E473740293686017
:061D8F00EFA3A3A380DF17
:061D95008A838982E473D9
:101D9B00EF4E6012EF60010EEDBB010B89828A835F
:101DAB00F0A3DFFCDEFA2289F05007F709DFFCA96C
:0C1DBB00F022BBFEFCF309DFFCA9F022C3
:00000001FF
